:100000000C943E050C9485050C948A060C94850589
:100010000C9485050C9485050C9485050C94850538
:100020000C9485050C9485050C94710D0C94430E6D
:100030000C942E1D0C9485050C9485050C94850557
:100040000C9485050C9485050C9485050C94850508
:100050000C9485050C94A21D0C9485050C948505C3
:100060000C9485050C9485050C9485050C948505E8
:100070000C9485050C9485050C9485050C948505D8
:100080000C9485050C9485050C9485050C948505C8
:100090000C9485050C9485050C9485050C948505B8
:1000A0000C9485050C9485050C948505A507B80767
:1000B000D107D507D907DC07E207E607EA07EE070D
:1000C000F207B00ED20EC00FD20EC00F170F3A0FAC
:1000D000C00F8F0FA20FF712F712261326138413E7
:1000E000C213DC15DC15DB13DC15DC14DC14B015D5
:1000F000DC15DC15C71500291E1F2021222324250D
:1001000026272D2E2A2B141A0815171C180C12132B
:100110002F3028E0041607090A0B0D0E0F33343573
:10012000E1311D1B0619051110363738E555E22C53
:10013000393A3B3C3D3E3F4041424353475F60615B
:10014000565C5D5E57595A5B626358E4544445E619
:10015000ABE3E765A5A6A8B4B0A7AFB6BCBBBAB978
:10016000B8B5B3B2AC4A524BAA50A94FB74D514E95
:10017000494C46480000706275663A2066756C6CA2
:100180000A002530325820004B6579626F61726435
:100190002073746172742E0A0055534220636F6E8F
:1001A000666967757265642E0A000D0A696E697466
:1001B0000A005B445D005B435D002C035800540063
:1001C00020006B006500790062006F006100720022
:1001D0006400200063006F006E007600650072000E
:1001E00074006500720000000E0374002E006D00A4
:1001F0002E006B002E0000000403090409028D008C
:10020000050100A0320904000001030101000921D9
:10021000110100012240000705810308000A0904BA
:1002200001000103010200092111010001224D001A
:100230000705820308000A09040200010300000008
:100240000921110100012236000705830308000A75
:10025000090403000203000000092111010001222A
:100260002200070584032000010705040320000184
:10027000090404000103000000092111010001220A
:10028000390007058503200001120110010000005C
:1002900008EDFE126501000102000105010906A139
:1002A00001050719E029E715002501950875018169
:1002B0000205081901290595057501910295017539
:1002C0000391010507190029F71500250195F87517
:1002D000018102C00631FF0974A1010975150026CC
:1002E000FF009520750881020976150026FF00950C
:1002F0002075089102C005010980A10185021681BF
:100300000026B7001A81002AB700751095018100F8
:10031000C0050C0901A1018503160100269C021AE3
:1003200001002A9C02751095018100C00501090297
:10033000A1010901A10005091901290515002501DF
:10034000950575018102950175038101050109304B
:1003500009311581257F95027508810609381581B7
:10036000257F950175088106050C0A38021581253F
:100370007F950175088106C0C005010906A1010528
:100380000719E029E71500250195087501810295F7
:100390000175088101050819012905950575019167
:1003A000029501750391010507190029FF15002623
:1003B000FF00950675088100C0636F6E73756D65EB
:1003C000723A20253034580A0073797374656D3A97
:1003D00020253034580A000A002530325820006B9E
:1003E0006579626F6172643A20004C45443A202579
:1003F0003032580A00253032583A202530386225EC
:10040000730A00722F632030313233343536370AA5
:100410000064656C5F6B65795F6269743A20636143
:100420006E27742064656C3A20253032580A0061CA
:1004300064645F6B65795F6269743A2063616E27FB
:1004400074206164643A20253032580A00290A0079
:100450002575002F002575005D280025640020000B
:10046000256400200025640020002564007C002510
:10047000303258006D6F7573656B6579205B6274FF
:100480006E7C782079207620685D287265702F61F7
:10049000636C293A205B006D6B5F776865656C5F04
:1004A00074696D655F746F5F6D6178203D202564B0
:1004B0000A006D6B5F776865656C5F6D61785F736F
:1004C00070656564203D2025640A006D6B5F74696A
:1004D0006D655F746F5F6D6178203D2025640A0053
:1004E0006D6B5F6D61785F7370656564203D20257D
:1004F000640A006D6B5F696E74657276616C203D95
:100500002025640A006D6B5F64656C6179203D2075
:1005100025640A006D6B5F776865656C5F74696D53
:10052000655F746F5F6D6178203D2025640A006D02
:100530006B5F776865656C5F6D61785F737065652B
:1005400064203D2025640A006D6B5F74696D655FF2
:10055000746F5F6D6178203D2025640A006D6B5FCC
:100560006D61785F7370656564203D2025640A00C5
:100570006D6B5F696E74657276616C203D202564D9
:100580000A006D6B5F64656C6179203D2025640A0B
:10059000000A00257500363A20776865656C5F743F
:1005A000696D655F746F5F6D61783A20000A0025A0
:1005B0007500353A20776865656C5F6D61785F73AB
:1005C000706565643A20000A00257500343A20748D
:1005D000696D655F746F5F6D61783A20000A002570
:1005E0007500333A206D61785F73706565643A20F9
:1005F000000A00257500323A20696E7465727661D2
:100600006C286D73293A20000A00257500313A20C4
:1006100064656C6179282A31306D73293A20000AAB
:10062000092D2056616C756573202D0A004D3E0022
:100630004D25643E20003F0073657420646566614B
:10064000756C740A00433E2000776865726520640B
:10065000656C74613A20637572736F723D25642C0A
:1006600020776865656C3D25640A5365652068746C
:1006700074703A2F2F656E2E77696B6970656469A7
:10068000612E6F72672F77696B692F4D6F75736578
:100690005F6B6579730A000A092D204D6F757365CC
:1006A0006B6579202D0A4553432F713A097175699D
:1006B000740A313A0964656C6179282A31306D73A6
:1006C000290A323A09696E74657276616C286D7315
:1006D000290A333A096D61785F73706565640A347D
:1006E0003A0974696D655F746F5F6D61780A353AB8
:1006F00009776865656C5F6D61785F7370656564C7
:100700000A363A09776865656C5F74696D655F7470
:100710006F5F6D61780A0A703A097072696E7420B1
:1007200076616C7565730A643A0973657420646553
:100730006661756C74730A75703A092B310A646FBF
:10074000776E3A092D310A706775703A092B31308E
:100750000A7067646F776E3A092D31300A0A737038
:10076000656564203D2064656C7461202A206D619C
:10077000785F7370656564202A20287265706561F2
:1007800074202F2074696D655F746F5F6D617829C7
:100790000A003F004D3E2000433E20004C25640AE5
:1007A000000A092D20436F6E736F6C65202D0A457A
:1007B00053432F713A09717569740A6D3A096D6F67
:1007C0007573656B65790A000A092D204D616769AB
:1007D00063202D0A643A0964656275670A783A09EC
:1007E0006465627567206D61747269780A6B3A0995
:1007F0006465627567206B6579626F6172640A6D0A
:100800003A096465627567206D6F7573650A763A9B
:100810000976657273696F6E0A733A09737461744D
:1008200075730A633A09636F6E736F6C65206D6F41
:1008300064650A302D343A096C61796572302D3463
:10084000284631302D4634290A506175733A0962C1
:100850006F6F746C6F616465720A6E3A094E4B5229
:100860004F0A003F004E4B524F3A206F66660A0017
:100870004E4B524F3A206F6E0A0074696D65725F7D
:1008800072656164333228293A202530346C580A65
:10089000006B6579626F6172645F6E6B726F3A2094
:1008A00025580A006B6579626F6172645F69646CD8
:1008B000653A2025580A006B6579626F6172645F42
:1008C00070726F746F636F6C3A2025580A00686FFE
:1008D00073745F6B6579626F6172645F6C6564737A
:1008E00028293A2025580A000A092D2053746174DA
:1008F0007573202D0A004743433A20342E392E3297
:10090000204156522D4C4942433A20312E382E3048
:1009100073766E204156525F415243483A206176C9
:1009200072350A004F5054494F4E533A204C5546A9
:1009300041204D4F5553454B455920455854524140
:100940004B455920434F4E534F4C4520434F4D4D3F
:10095000414E44204E4B524F203531320A00425511
:10096000494C443A20653131333433342028323114
:100970003A34363A3332204D6172203134203230ED
:100980003138290A005649443A20307846454544D2
:1009900028742E6D2E6B2E29205049443A20307831
:1009A00036353132285854206B6579626F61726434
:1009B00020636F6E76657274657229205645523ACF
:1009C000203078303030310A00444553433A2063B8
:1009D0006F6E76657274205854206B6579626F6112
:1009E000726420746F205553420A000A092D205664
:1009F000657273696F6E202D0A000A6D6F757365DD
:100A00003A206F66660A000A6D6F7573653A206F4B
:100A10006E0A000A6B6579626F6172643A206F66D4
:100A2000660A000A6B6579626F6172643A206F6EC4
:100A30000A000A6D61747269783A206F66660A006E
:100A40000A6D61747269783A206F6E0A000A6465F3
:100A50006275673A206F6E0A000A64656275673ACC
:100A6000206F66660A000A0A626F6F746C6F6164B9
:100A700065722E2E2E2000433E20000011241FBE42
:100A8000CFEFDAE0DEBFCDBF04B603FE27C0809112
:100A9000CF029091D002A091D102B091D2028730C2
:100AA000904BA740B04BD1F41092CF021092D002DD
:100AB0001092D1021092D20214BE84B7877F84BFF5
:100AC0000FB6F894A89580916000886180936000CB
:100AD000109260000FBEE0E0FFE3099511E0A0E096
:100AE000B1E0EEE8FDE402C005900D92A833B10735
:100AF000D9F722E0A8E3B1E001C01D92AF3CB207F4
:100B0000E1F70E94940A0C94C5260C940000FF9310
:100B1000EF93E0913801F0913901309709F0099590
:100B2000EF91FF910895FC018591803011F0EFDF86
:100B3000FBCF0895FF27E0E230E247FF0CC041956C
:100B400097FF09C0EDE26095709580959095611DC5
:100B5000711D811D911D27FF02C0219530E350E2D8
:100B6000AA27660F771F881F991FAA1FA41710F0C6
:100B7000A41B63955A95A9F7AA3008F0A95FA05D58
:100B8000AF93F395611571058105910541F7ED323C
:100B900011F4EF93F395F21718F43F93F395FBCF0D
:100BA0008F91B5DFFA95E1F70895E991F991859173
:100BB000803021F0853219F0AADFF9CF089520E0C6
:100BC000E89455915532C1F3503311F4689455911E
:100BD0005A3348F4505390F3220F022E220F220F63
:100BE000200D250FF4CF0EF421958991999153365C
:100BF00019F3533729F1533559F1BC018827992747
:100C0000E8945C3621F48991999168945591543611
:100C100039F446EF7EF077FF0DC08FEF9FEF0AC0EB
:100C200055374AE039F0583540E121F0523642E07C
:100C300009F00895FF93EF937DDFEF91FF91B7CF18
:100C4000FF93EF93FC0181918030B9F360DFFBCF1C
:100C5000FF93EF9368DFF1CFDF93CF93CDB7DEB78C
:100C60002596A3DFCF91DF910895E9E6F0E080813A
:100C700088608083E9982F98279A2FEF89E698E17A
:100C8000215080409040E1F700C00000279858981C
:100C9000509A5998519A2FEF89EF90E02150804057
:100CA0009040E1F700C000005198599A5098589A26
:100CB000E19AE99A08954FB7F89420913E01309156
:100CC0003F0180913C0190913D014FBF28173907AA
:100CD000F9F09FB7F89420913C0130913D0140918B
:100CE0003E0150913F014217530779F0F901EE0F91
:100CF000FF1FE05CFE4F80812F5F3F4F2F71332736
:100D000030933D0120933C0101C080E09FBF0895D6
:100D100080E008951F920F920FB60F9211242F9327
:100D20003F934F935F936F937F938F939F93AF9373
:100D3000BF93CF93EF93FF9329B1217090913B0123
:100D4000992319F0993058F403C0211108C037C015
:100D500080913A0186952111806880933A0181E063
:100D6000890F80933B01983051F540913A0150E052
:100D7000CFB7F89480913E0190913F019C012F5F85
:100D80003F4F2F71332760913C0170913D01261731
:100D9000370761F0880F991FFC01E05CFE4F51831B
:100DA000408330933F0120933E0104C086E791E0E9
:100DB0000E949305CFBF10923B0110923A01FF9120
:100DC000EF91CF91BF91AF919F918F917F916F9153
:100DD0005F914F913F912F910F900FBE0F901F90F9
:100DE0001895803389F1A0F48E3138F48C3140F5B8
:100DF000803181F1893111F10895843219F128F49B
:100E000090EE980F9330F0F008958E32E9F0089547
:100E10008A3448F48734E0F48533C1F08833B1F084
:100E20008233C9F411C08D3499F018F48B3481F0F9
:100E3000089591EB980F953058F008958AE508953C
:100E4000885C0895805C08958C5B08958F5D08959B
:100E5000885D08958EE60895CF93DF93D82FD770DD
:100E6000C82FC695C695C6956D2F8C2F0E9445112B
:100E7000882371F0EC2FF0E0EF57FE4F81E090E017
:100E800001C0880FDA95EAF78095908189238083E5
:100E9000DF91CF910895CF93DF93D82FD770C82FCC
:100EA000C695C695C6956D2F8C2F0E944511811150
:100EB0000DC0EC2FF0E0EF57FE4F81E090E001C055
:100EC000880FDA95EAF79081892B8083DF91CF91A3
:100ED00008958091B10281608093B1020E9435062D
:100EE000E1E8F1E080E18E0F11928E13FDCF0895BD
:100EF000CF93DF931F92CDB7DEB765E08FE00E94FE
:100F00004511882319F08DE70E942C070E945B068B
:100F1000882371F01F928F9322E831E03F932F9343
:100F200089830E942C060F900F900F900F9089815B
:100F3000E09180014E2F50E04B30510508F058C031
:100F4000FA01EA5AFF4F0C94AB26803E21F0813E15
:100F500021F486E014C081E012C01816BCF09FE7AF
:100F6000980F9E3708F044C080580E942C0740C05C
:100F70008A3221F0873B31F484E001C082E0809323
:100F8000800138C018162CF40E94F1060E944B070D
:100F90002FC09FE7980F9E3758F580580E94F106A2
:100FA000E4CF803E29F583E0EACF873309F58CE76B
:100FB0001CC0803EE9F41EC08A3AD1F48CE70E943E
:100FC0002C0718C08D31A1F487E0D9CF853481F486
:100FD00088E0D5CF813E61F489E0D1CF8D3941F4ED
:100FE0008AE0CDCF853C21F48DE70E944B0702C0FB
:100FF0001092800181E00F90DF91CF910895E82F4A
:10100000F0E0EF57FE4F80810895E1E8F1E080E1E4
:101010008E0F11928E13FDCF089508958091B50122
:1010200008959FB7F894109294019FBF9091C602C3
:10103000943009F057C09091E9009F703091EC0016
:10104000232F217030FD20E8922B24E02093E9002B
:101050002091EB0020FF43C02091EE0027FF3FC00E
:1010600020919101222321F02091E80025FF37C033
:101070001092910126E03091E80035FD15C03091C5
:10108000C602343061F53091EB0035FD28C02150A7
:1010900021F481E08093910122C0EFE9FFE03197D4
:1010A000F1F700C00000E7CF8093F1008091E800E5
:1010B00085FD0AC08091E80080FFFCCF8091E800A8
:1010C0008E778093E80006C08FB7F89421E02093D4
:1010D00094018FBF9F709093E90080E008959F7006
:1010E0009093E9008FEF0895CF93DF9300D01F9284
:1010F000CDB7DEB79C018091C602843019F593E02C
:1011000099833B832A839093E9008FEF9091E800C5
:10111000815095FD06C095ED9A95F1F7000081117B
:10112000F5CF8091E80085FF0DC040E050E063E01E
:1011300070E0CE0101960E94610B8091E8008E77ED
:101140008093E8000F900F900F90DF91CF9108955A
:10115000CF93DF9300D01F92CDB7DEB72091C602A8
:10116000243021F522E029839B838A8383E08093C6
:10117000E9008FEF9091E800815095FD06C095ED54
:101180009A95F1F700008111F5CF8091E80085FF75
:101190000DC040E050E063E070E0CE0101960E9497
:1011A000610B8091E8008E778093E8000F900F909C
:1011B0000F90DF91CF9108952091C6022430F1F471
:1011C00022E02093E9002FEF3091E800215035FD17
:1011D00006C035ED3A95F1F700002111F5CF2091C9
:1011E000E80025FF0BC040E050E065E070E00E94A1
:1011F000610B8091E8008E778093E8000895CF938B
:10120000DF932091C602243009F048C0EC018091A0
:101210000A018823E1F080910B018823C1F085E069
:101220008093E9008FEF9091E800815095FD06C012
:101230009AE29A95F1F700C08111F5CF8091E8000C
:1012400085FF2CC040E050E060E270E017C081E014
:101250008093E9008FEF9091E800815095FD06C0E2
:1012600095ED9A95F1F700008111F5CF8091E80096
:1012700085FF14C040E050E068E070E0CE010E94BD
:10128000610B8091E8008E778093E80080E2FE0198
:10129000A5E9B1E001900D928A95E1F7DF91CF9138
:1012A000089586EB91E00E9493058091C50281111B
:1012B00009C00E94F60C0E94530D8091E2008460E8
:1012C0008093E200089582EB91E00E9493051092D2
:1012D000C50208950895209192012F5F822F62E345
:1012E0000E948B26992319F0209392010895109261
:1012F000920180919401882371F18091C60284301B
:1013000041F58091E9008F702091EC00922F91704F
:1013100020FD90E8892B94E09093E9009091EB00F8
:1013200090FF14C09091EE0097FF10C09091E800DC
:1013300095FF03C01092F100F9CF9091E80090FF63
:1013400005C09091E8009E779093E8008F7080939D
:10135000E90010929401089542E061EC81E00E945E
:10136000700C42E061EC82E00E94700C42E061ECA3
:1013700083E00E94700C42E261EC84E00E94700CF9
:1013800042E261EC85E00C94700C8091C8028330DD
:1013900009F455C030F4813071F0823009F48EC008
:1013A00008958A3009F47AC08B3009F460C089301E
:1013B00009F09CC020C08091C702813A09F096C014
:1013C0008091E800877F8093E8008091CB02909124
:1013D000CC02892B21F460E285E991E003C060E052
:1013E00080E090E070E00E94AC0B8091E8008B7789
:1013F0008093E80008958091C702813209F076C099
:101400008091CB029091CC02009719F0049709F0DB
:101410006DC08091E800877F8093E8008091E800AC
:1014200082FD05C08091C6028111F8CF5FC0809116
:10143000F1008093B5018091E8008B7753C08091D3
:10144000C702813A09F052C08091CB029091CC0240
:10145000892B09F04BC08091E800877F8093E800DA
:101460008091E80080FFFCCF80910A0136C0809116
:10147000C7028132D9F58091CB029091CC02892BA1
:10148000A9F58091E800877F8093E8000E94A50C71
:101490008091C90280930A010C94FE158091C702C5
:1014A000813221F58091E800877F8093E8000E94D7
:1014B000A50C8091CA028093B60108958091C7025D
:1014C000813AA1F48091E800877F8093E8008091C1
:1014D000E80080FFFCCF8091B6018093F1008091FD
:1014E000E8008E778093E8000C94A50C0895089589
:1014F00008958091B501809393011092B50180E029
:101500000E940D080E9405080C94FE150C94790A9F
:101510000E94ED1C8091C402882329F00E94161DB0
:1015200081110C944B0B089584B7877F84BF0FB64D
:10153000F894A89580916000886180936000109273
:1015400060000FBE90E080E80FB6F89480936100D1
:10155000909361000FBE81E198E00E94BE1C8AEA70
:1015600091E00E9493050E94770A0E9499100E94C0
:10157000F60C0E94530D8091E20084608093E2009B
:1015800078948091C6028430E1F781ED97E001976D
:1015900039F0EFE9FFE03197F1F700C00000F7CF35
:1015A00089E991E00E9493050E949B1080E091E000
:1015B0000E94D80F88E891E00E9493050E94780A63
:1015C0008091C602853019F40E94880AF9CF0E94E2
:1015D0009F10F6CF0E942A1D809193018093B50140
:1015E00008950C94EA0A292F332723303105C9F0D6
:1015F00064F42130310581F02230310509F043C017
:101600008DE890E02CEF31E042C021323105F1F05D
:101610002232310541F137C082E190E029E832E021
:1016200036C099278130910541F08230910541F013
:10163000892B49F5E8EFF1E005C0E8EEF1E002C0E2
:10164000EAEBF1E0849190E09F0121C06530D8F48D
:10165000E62FF0E0EE0FFF1FED5DFE4F20813181A0
:1016600089E090E014C0653070F470E0FB01EE0F8B
:10167000FF1FE75EFE4F20813181FB01EC5EFE4FD4
:10168000808190E004C080E090E020E030E0FA014A
:1016900031832083089580E189BD82E189BD09B449
:1016A00000FEFDCF8091D8008F7D8093D80080917F
:1016B000E00082608093E0008091E00081FDFCCF3B
:1016C0000895CF92DF92EF92FF920F931F93CF93E3
:1016D000DF93EC018B016A010E94C40C811133C0BD
:1016E000C114D10439F0F60180819181081B190BD6
:1016F000C80FD91FE12CF12C0115110519F18091AA
:10170000E80085FD16C08091E8008E778093E800A0
:10171000C114D10449F0F60180819181E80EF91ECF
:10172000F182E08285E00FC00E94C40C882321F37F
:101730000AC089918093F10001501109FFEFEF1A5F
:10174000FF0ADACF80E0DF91CF911F910F91FF90D8
:10175000EF90DF90CF9008952091CD023091CE028E
:101760002617370748F06115710539F42091E80014
:101770002E772093E80001C0B90140E061157105A2
:10178000A9F12091C602222309F443C0253009F4AF
:1017900042C02091E80023FD40C02091E80022FDD6
:1017A00032C02091E80020FFE9CF4091F300209162
:1017B000F20030E0342BFC01CF016115710559F0C6
:1017C0002830310540F481918093F1006150710916
:1017D0002F5F3F4FF1CF41E02830310509F040E065
:1017E0002091E8002E772093E800C8CF4111C9CF9F
:1017F0000AC08091C602882361F0853061F0809133
:10180000E80083FD0AC08091E80082FFF2CF80E00B
:10181000089582E0089583E0089581E0089520917D
:10182000CD023091CE022617370748F061157105B9
:1018300039F42091E8002E772093E80001C0B90127
:10184000FC0120E06115710591F18091C6028823A9
:1018500009F440C0853009F43FC08091E80083FD61
:101860003DC08091E80082FD2FC08091E80080FF9C
:10187000E9CF2091F3008091F20090E0922B611566
:10188000710559F08830910540F424912093F100BE
:101890003196615071090196F2CF21E0089709F065
:1018A00020E08091E8008E778093E800CBCF211173
:1018B000CCCF0AC08091C602882361F0853061F0E8
:1018C0008091E80083FD0AC08091E80082FFF2CF9A
:1018D00080E0089582E0089583E0089581E008950E
:1018E000982F973058F59093E900981739F0709138
:1018F000EC002091ED005091F00003C0242F762FD2
:1019000050E021FF19C03091EB003E7F3093EB0097
:101910003091ED003D7F3093ED003091EB00316070
:101920003093EB007093EC002093ED005093F000A7
:101930002091EE0027FF07C09F5FD3CF8F70809369
:10194000E90081E0089580E008958091C70287FF53
:1019500011C08091E80082FD05C08091C60281110E
:10196000F8CF11C08091E8008B770BC08091C60240
:10197000882349F08091E80080FFF8CF8091E8004B
:101980008E778093E80008952091E4003091E5007F
:1019900095E64091EC00842F817040FF22C0809139
:1019A000E80080FD1CC08091C602882391F085303C
:1019B00091F08091EB0085FD10C04091E4005091C2
:1019C000E5004217530729F39A01915011F784E07B
:1019D000089582E0089583E0089581E0089580E00D
:1019E00008954091E80042FFDECF08950E94640D03
:1019F0000E946C0DE0EEF0E0808181608083E8ED74
:101A0000F0E080818F77808319BCA7EDB0E08C91E6
:101A10008E7F8C9380818F7E80831092C502089583
:101A20000F931F93CF93DF930E94640D0E946C0D60
:101A3000C8EDD0E088818F7788838881806888832B
:101A400088818F7D888319BC1092C6021092C202D1
:101A50001092C4021092C30200EE10E0F8018081DF
:101A60008B7F808388818160888342E060E080E0B2
:101A70000E94700CE1EEF0E080818E7F8083E2EEC8
:101A8000F0E0808181608083808188608083F801BC
:101A900080818E7F8083888180618883DF91CF9170
:101AA0001F910F910895E8EDF0E080818F7E808393
:101AB000E7EDF0E080818160808384E082BF81E097
:101AC0008093C5020C94100DE8EDF0E080818E7FCC
:101AD00080831092E20008951092DA001092E100E3
:101AE00008951F920F920FB60F9211242F933F93D8
:101AF0004F935F936F937F938F939F93AF93BF9316
:101B0000EF93FF938091E10082FF0BC08091E20090
:101B100082FF07C08091E1008B7F8093E1000E94EB
:101B20006B098091DA0080FF1FC08091D80080FF90
:101B30001BC08091DA008E7F8093DA008091D900FB
:101B400080FF0DC080E189BD82E189BD09B400FE3E
:101B5000FDCF81E08093C6020E94510905C019BCE7
:101B60001092C6020E9463098091E10080FF19C0B3
:101B70008091E20080FF15C08091E2008E7F80930B
:101B8000E2008091E20080618093E2008091D800C1
:101B900080628093D80019BC85E08093C6020E94C1
:101BA000860A8091E10084FF30C08091E20084FFCA
:101BB0002CC080E189BD82E189BD09B400FEFDCF62
:101BC0008091D8008F7D8093D8008091E1008F7E36
:101BD0008093E1008091E2008F7E8093E20080910B
:101BE000E20081608093E2008091C202882311F0BC
:101BF00084E007C08091E30087FD02C081E001C05E
:101C000083E08093C6020E94F10A8091E10083FF85
:101C100029C08091E20083FF25C08091E100877F89
:101C20008093E10082E08093C6021092C20280910C
:101C3000E1008E7F8093E1008091E2008E7F8093AF
:101C4000E2008091E20080618093E20042E060E087
:101C500080E00E94700C8091F00088608093F0001A
:101C60000E946A09FF91EF91BF91AF919F918F916F
:101C70007F916F915F914F913F912F910F900FBE88
:101C80000F901F9018951F920F920FB60F9211246C
:101C90002F933F934F935F936F937F938F939F9374
:101CA000AF93BF93CF93DF93EF93FF93C091E9007E
:101CB000CF708091EC00D82FD17080FDD0E81092C9
:101CC000E9008091F000877F8093F00078940E9473
:101CD000870E1092E9008091F00088608093F000F8
:101CE000CD2BCF70C093E900FF91EF91DF91CF91A1
:101CF000BF91AF919F918F917F916F915F914F9124
:101D00003F912F910F900FBE0F901F9018951F932A
:101D1000CF93DF93CDB7DEB7AA970FB6F894DEBFA7
:101D20000FBECDBFE7ECF2E088E08E0F9091F1009E
:101D300091938E13FBCF0E94C5098091E80083FF29
:101D40001FC18091C7029091C802492F50E04A30CC
:101D5000510508F015C1FA01EF59FF4F0C94AB265D
:101D6000803881F0823809F00BC18091CB028F70EE
:101D70008093E9008091EB0085FB882780F9109221
:101D8000E90006C08091C3029091C4029111826063
:101D90009091E800977F9093E8008093F100109273
:101DA000F100C8C0282F2D7F09F0EAC0882319F060
:101DB000823061F0E5C08091C902813009F0E0C055
:101DC000933009F080E08093C4022BC08091C90257
:101DD000811127C08091CB028F7009F4D1C080930C
:101DE000E9002091EB0020FF1CC0933021F480918A
:101DF000EB00806214C09091EB0090619093EB0037
:101E000021E030E0A90102C0440F551F8A95E2F796
:101E10004093EA001092EA008091EB008860809382
:101E2000EB001092E9008091E800877F86C0811165
:101E3000A7C01091C9021F778091E3008078812BA1
:101E40008093E3008091E800877F8093E8000E9400
:101E5000A50C8091E80080FFFCCF8091E3008068B2
:101E60008093E300111102C082E001C083E08093FF
:101E7000C60286C08058823008F082C08091C902B4
:101E80009091CA028C3D53E0950779F583E08A83EF
:101E90008AE289834FB7F894DE01139620E03EE092
:101EA00051E2E32FF0E050935700E49120FF03C08C
:101EB000E295EF703F5FEF708E2F90E0EA3010F008
:101EC000C79601C0C0968D939D932F5F243149F72B
:101ED0004FBF8091E800877F8093E8006AE270E05E
:101EE000CE0101960E94AC0B14C0AE014F5F5F4F54
:101EF0006091CB020E94F30ABC01892B09F440C017
:101F00009091E800977F9093E80089819A810E94E0
:101F10000F0C8091E8008B778093E80031C0803807
:101F200079F58091E800877F8093E8008091C20274
:101F30008093F1008091E8008E778093E8000E9402
:101F4000A50C1EC081111CC09091C9029230C0F432
:101F50008091E800877F8093E8009093C2020E94FE
:101F6000A50C8091C202811106C08091E30087FD1B
:101F700002C081E001C084E08093C6020E94AC09E7
:101F80008091E80083FF0AC08091E800877F8093FA
:101F9000E8008091EB0080628093EB00AA960FB678
:101FA000F894DEBF0FBECDBFDF91CF911F91089592
:101FB0009093BC018093BB010895E091BB01F09127
:101FC000BC01309721F00190F081E02D099480E070
:101FD0000895EF92FF920F931F93CF93DF93E091B9
:101FE000BB01F091BC013097B1F18C010280F3810B
:101FF000E02D09958091B10282FF2DC080FF04C0C1
:102000008FED93E00E949305E80110E289EDE82E40
:1020100083E0F82E8091B10280FF0BC088811F926F
:102020008F93FF92EF920E942C060F900F900F90CB
:102030000F90115021961111EDCF8091B10280FFC8
:102040000AC087ED93E0DF91CF911F910F91FF9030
:10205000EF900C949305DF91CF911F910F91FF901A
:10206000EF900895E091BB01F091BC01309721F011
:102070000480F581E02D09940895CF93DF93EC015E
:102080008091B9019091BA01C817D90709F1D0938D
:10209000BA01C093B901E091BB01F091BC01309746
:1020A000B9F00680F781E02DCE0109958091B1024B
:1020B00082FF0EC080FF0CC0DF93CF9389EC93E0CA
:1020C0009F938F930E942C060F900F900F900F906C
:1020D000DF91CF910895CF93DF93EC018091B70109
:1020E0009091B801C817D90709F1D093B801C093EE
:1020F000B701E091BB01F091BC013097B9F00084C9
:10210000F185E02DCE0109958091B10282FF0EC0CC
:1021100080FF0CC0DF93CF9389EB93E09F938F9365
:102120000E942C060F900F900F900F90DF91CF918F
:1021300008950C9444110E94571D0C946907BF9296
:10214000CF92DF92EF92FF920F931F93CF93DF9383
:1021500000D000D01F92CDB7DEB70E9478070EEBFB
:1021600011E0F12C8F2D0E94FF07B82EF801C080DE
:10217000C82639F4F3940F5F1F4FF0E1FF12F2CF3E
:1021800030C08091B10281FD0E946011D12CEE24FB
:10219000E3948E2D8C21F9F0D982FA8281E09E2D74
:1021A0009B2109F480E08B830E94601D8160782F61
:1021B0009D838C8349815A816B818D810E94961108
:1021C00049815A816B817C818D810E94DA1CF801E2
:1021D00090819E259083D394EE0CF8E0DF12D9CF46
:1021E000C9CF8FEF89838A831B820E94601D816023
:1021F000782F9D838C8349815A816B818D810E94C8
:1022000096110E94D91C0E94B9201091BD010E9414
:10221000DD0F181741F10E94DD0F8093BD019091F1
:10222000B10292FF0EC090FF0CC01F928F938AEEF6
:1022300093E09F938F930E942C060F900F900F9026
:102240000F908091BD010F900F900F900F900F9005
:10225000DF91CF911F910F91FF90EF90DF90CF9082
:10226000BF900C94EB1C0F900F900F900F900F905D
:10227000DF91CF911F910F91FF90EF90DF90CF9062
:10228000BF9008950C940D080895CF93DF931F928B
:10229000CDB7DEB769830E94FF0790E021E030E010
:1022A000698102C0220F331F6A95E2F72823392380
:1022B00081E0232B09F480E00F90DF91CF91089506
:1022C000EF92FF920F931F93CF93DF9383E094E0FD
:1022D0000E949305C0E0D0E08DE2E82E81E0F82E68
:1022E00005EF13E08C2F0E94FF070E94C31CFF9292
:1022F000EF921F928F93DF93CF931F930F930E94C0
:102300002C0621968DB79EB708960FB6F8949EBFFF
:102310000FBE8DBFC031D10529F7DF91CF911F913D
:102320000F91FF90EF90089508950895CF93DF9354
:10233000CDB7DEB72B970FB6F894DEBF0FBECDBF7B
:10234000942F4F83252F588769877A878B874A85F3
:102350005B85452B21F02F3F09F59F3FF9F4DE0106
:10236000119686E0FD0111928A95E9F785E0FE015C
:10237000379601900D928A95E1F749815A816B81D8
:102380007C818D819E810E94DB182B960FB6F8947C
:10239000DEBF0FBECDBFDF91CF9108954F8158852D
:1023A00069857A858B850E94DA1CD9CFCF938823E3
:1023B00009F4A4C0C82F8CEF8C0F813A48F48C2FFD
:1023C0000E94032481119AC08C2F0E94B31B0CC061
:1023D00080E28C0F883058F4C77081E001C0880F0C
:1023E000CA95EAF70E945E1CCF910C94981C8BE56D
:1023F0008C0F833078F4C53A29F0C63A31F083E87F
:1024000090E005C081E890E002C082E890E0CF91C2
:102410000C943D1088E58C0F853108F06FC0C83AE8
:1024200061F1C93A69F1CA3A71F1CB3A79F1CC3A22
:1024300081F1CD3A89F1CE3A91F1CF3A99F1C13B90
:10244000A1F1C03BA9F1C23BB1F1C33BB9F1C43B1F
:10245000C1F1C53BC9F1C63BD1F1C73BD9F1C83B7E
:10246000E1F1C93BE9F1CA3BF1F1CB3BF9F1CC3BDE
:1024700009F43FC080E090E03EC082EE90E03BC0B7
:1024800089EE90E038C08AEE90E035C085EB90E0B0
:1024900032C086EB90E02FC083EB90E02CC084EB41
:1024A00090E029C087EB90E026C08CEC90E023C040
:1024B0008DEC90E020C083E891E01DC08AE891E0B7
:1024C0001AC082E991E017C084E991E014C081E26A
:1024D00092E011C083E292E00EC084E292E00BC071
:1024E00085E292E008C086E292E005C087E292E0D1
:1024F00002C08AE292E0CF910C946B10CF910895C4
:10250000882329F19CEF980F913A18F40E94061C39
:102510000DC090E2980F983058F4877091E001C098
:10252000990F8A95EAF7892F0E94641C0C94981CD5
:102530009BE5980F933020F480E090E00C943D10E0
:10254000885A853120F480E090E00C946B10089557
:10255000882321F00E945E1C0C94981C0895882307
:1025600021F00E94641C0C94981C0895BF92CF9295
:10257000DF92EF92FF920F931F93CF93DF9300D0E0
:1025800000D000D0CDB7DEB725E0FC01DE0111960A
:1025900001900D922A95E1F7FC0140815181028161
:1025A00063817481258122952F706115710509F46D
:1025B00003C35F3F19F44F3F09F4FEC26C01862F3D
:1025C0007D836C83602F782F8D812E830E94371B33
:1025D000182FB92E0E94361B0E94261AEB2DE29569
:1025E000EF70F0E0E559FF4F2E810C94AB268B2D58
:1025F000807F9B2D9F70F92E882319F0F29490EF25
:10260000F922002349F0FF2009F483C28F2D0E9494
:10261000711C0E94981C7DC2812F0E948012FF2095
:1026200009F4CAC28F2D0E94771C26960FB6F89423
:10263000DEBF0FBECDBFDF91CF911F910F91FF90F5
:10264000EF90DF90CF90BF900C94981C8B2D807FE3
:102650009B2D9F70F92E803219F0F29480EFF822B2
:10266000112319F0113009F12AC00023B1F08F2D88
:10267000222351F1213041F526960FB6F894DEBFA2
:102680000FBECDBFDF91CF911F910F91FF90EF90C3
:10269000DF90CF90BF900C94811C222319F0213041
:1026A00009F48AC20E94841C2DC00023F1F0263058
:1026B00008F082C20E945B1C8F2129F023C00023F6
:1026C000F9F0211116C08F2D26960FB6F894DEBFB3
:1026D0000FBECDBFDF91CF911F910F91FF90EF9073
:1026E000DF90CF90BF900C94A812253008F064C200
:1026F00009C0F601858180FF0CC28F708583E3CF0E
:1027000021111CC28F2D83C12B2D26952695237058
:1027100030E02115310521F021303105D1F04CC2D6
:10272000002321F0812F9B2D937002C080E090E068
:1027300026960FB6F894DEBF0FBECDBFDF91CF91C6
:102740001F910F91FF90EF90DF90CF90BF900C946E
:102750003D10002321F0812F9B2D937002C080E05B
:1027600090E026960FB6F894DEBF0FBECDBFDF9186
:10277000CF911F910F91FF90EF90DF90CF90BF907E
:102780000C946B10812F002319F00E943F1F02C090
:102790000E94A71F26960FB6F894DEBF0FBECDBFCE
:1027A000DF91CF911F910F91FF90EF90DF90CF902D
:1027B000BF900C942C208B2D837009F07BC00111ED
:1027C000FBC1812F829586958770880F880F912F86
:1027D0009F70C92ED12CE12CF12C082E04C0CC0CFA
:1027E000DD1CEE1CFF1C0A94D2F714FF12C04FE050
:1027F00050E060E070E004C0440F551F661F771F73
:102800008A95D2F7CB01BA01609570958095909525
:1028100003C060E070E0CB012B2D26952695237038
:10282000422F50E042305105D9F04330510569F153
:102830006C297D298E299F294130510551F1269619
:102840000FB6F894DEBF0FBECDBFDF91CF911F91C1
:102850000F91FF90EF90DF90CF90BF900C944B1AA8
:102860006C297D298E299F2926960FB6F894DEBF04
:102870000FBECDBFDF91CF911F910F91FF90EF90D1
:10288000DF90CF90BF900C94651A0E944B1AC7013D
:10289000B60126960FB6F894DEBF0FBECDBFDF910E
:1028A000CF911F910F91FF90EF90DF90CF90BF904D
:1028B0000C94311A002319F08B2D817001C086957C
:1028C000882309F479C1812F829586958770880FB6
:1028D000880F912F9F70C92ED12CE12CF12C082E3E
:1028E00004C0CC0CDD1CEE1CFF1C0A94D2F714FFB4
:1028F00012C04FE050E060E070E004C0440F551F8C
:10290000661F771F8A95D2F7CB01BA016095709543
:102910008095909503C060E070E0CB012B2D26954B
:1029200026952370422F50E042305105D9F04330B4
:10293000510569F16C297D298E299F294130510566
:1029400051F126960FB6F894DEBF0FBECDBFDF91D2
:10295000CF911F910F91FF90EF90DF90CF90BF909C
:102960000C94121B6C297D298E299F2926960FB65F
:10297000F894DEBF0FBECDBFDF91CF911F910F91B5
:10298000FF90EF90DF90CF90BF900C94241B0E949B
:10299000121BC701B60126960FB6F894DEBF0FBE14
:1029A000CDBFDF91CF911F910F91FF90EF90DF90FE
:1029B000CF90BF900C94001B103FD1F128F480E41D
:1029C000810F803250F0A0C0123F09F462C008F4B9
:1029D0004BC0133F09F472C097C0F12FF071FF2E66
:1029E0008B2D8F71002351F00E94991A812FFF20A7
:1029F00019F08295807F68CE8F7066CE0E94BA1AD9
:102A0000812FFF2019F08295807F01C08F7026965C
:102A10000FB6F894DEBF0FBECDBFDF91CF911F91EF
:102A20000F91FF90EF90DF90CF90BF900C94AF127A
:102A30000023B1F0253008F0BFC08B2D8F71269692
:102A40000FB6F894DEBF0FBECDBFDF91CF911F91BF
:102A50000F91FF90EF90DF90CF90BF900C94DF1A12
:102A6000263008F0A9C0E9CF0023A9F08B2D8F7183
:102A700026960FB6F894DEBF0FBECDBFDF91CF9183
:102A80001F910F91FF90EF90DF90CF90BF900C942B
:102A9000991A002359F38B2D8F7126960FB6F8944F
:102AA000DEBF0FBECDBFDF91CF911F910F91FF9081
:102AB000EF90DF90CF90BF900C94BA1A002399F05A
:102AC0008B2D8F7126960FB6F894DEBF0FBECDBF4B
:102AD000DF91CF911F910F91FF90EF90DF90CF90FA
:102AE000BF900C94841A26960FB6F894DEBF0FBEE2
:102AF000CDBFDF91CF911F910F91FF90EF90DF90AD
:102B0000CF90BF900C947F1A0023A9F0222309F4E0
:102B1000ADCF812F26960FB6F894DEBF0FBECDBF86
:102B2000DF91CF911F910F91FF90EF90DF90CF90A9
:102B3000BF900C94D611222309F4ADCF812F269695
:102B40000FB6F894DEBF0FBECDBFDF91CF911F91BE
:102B50000F91FF90EF90DF90CF90BF900C94801278
:102B60004B2D4F70612FC6010E94E91D26960FB6AE
:102B7000F894DEBF0FBECDBFDF91CF911F910F91B3
:102B8000FF90EF90DF90CF90BF900C947F194B2D6A
:102B90004F70612FC60126960FB6F894DEBF0FBEA8
:102BA000CDBFDF91CF911F910F91FF90EF90DF90FC
:102BB000CF90BF900C94EC1D26960FB6F894DEBF14
:102BC0000FBECDBFDF91CF911F910F91FF90EF907E
:102BD000DF90CF90BF9008950E947E1C0E944D1CF4
:102BE0000E94981C0E945E210E942C2080E090E0B0
:102BF0000E943D1080E090E00C946B100E946E1CCF
:102C00000C94EC15CF93DF9300D000D01F92CDB77A
:102C1000DEB7942F4983252F5A836B837C838D8362
:102C20004C815D81452B39F12F3F11F49F3F19F104
:102C300049815A816B817C818D810E94371B292FAC
:102C400022952F7030E02C30310504F52A30310503
:102C50005CF4225031092230310568F4853A80F461
:102C6000843090F4823080F0883E38F4803E60F406
:102C70008450813A48F080E014C0803FE1F704C0FE
:102C800090E2980F983080F781E00BC02C3031052E
:102C900021F493FB882780F904C02F303105C9F354
:102CA000EACF0F900F900F900F900F90DF91CF9180
:102CB0000895CF93DF9300D000D01F92CDB7DEB739
:102CC0000F900F900F900F900F90DF91CF9108957C
:102CD000CF93DF9300D000D000D0CDB7DEB72696DB
:102CE0000FB6F894DEBF0FBECDBFDF91CF91089530
:102CF0001F93CF93DF93C091CE0116E08091CF0157
:102D0000C81799F0D0E01C9FF0011D9FF00D112411
:102D1000E053FE4F408151816281738184819581AE
:102D20000E9468162196C770E9CFDF91CF911F915D
:102D30000895409100025091010260910202709149
:102D4000030280910402909105020C946816809110
:102D5000050282958F7009F054C080910202882389
:102D600009F44FC08091CE01A091CF016091000283
:102D7000709101024091030250910402B6E08A175B
:102D800009F43FC090E041155105C1F17F3F11F4B6
:102D90006F3FA1F1B89FF001B99FF00D1124E053EE
:102DA000FE4F218172132AC02081621327C0228125
:102DB000211124C0238134812417350710F42150B8
:102DC0003109241B350B283C3105C0F42091050244
:102DD0002F7020612093050226E0289FF001299F93
:102DE000F00D1124EB52FE4F80818F708061808343
:102DF00080E092E00E94B6120C94781601968770DB
:102E0000BECF0895BF92CF92DF92EF92FF920F93C1
:102E10001F93CF93DF93CDB7DEB761970FB6F894CA
:102E2000DEBF0FBECDBF7C0185E0F701DE011D9640
:102E300001900D928A95E1F7D7014C9111965C9122
:102E400011971296DC90129713960D911C9114977E
:102E5000309100026091010280910302909104027E
:102E6000009709F477C16F3F19F43F3F09F472C12D
:102E7000B0900202BB2009F4C5C0209105020817DA
:102E8000190728F0F801E81BF90BCF0104C0809561
:102E90009095800F911FCC24C394883C910580F0BD
:102EA000C12C207F09F0CCC0702F198B088B6D2DA1
:102EB00089890E94591680E092E00E94B612B6C03D
:102EC000822F807F09F047C0651314C0341312C0ED
:102ED000D11010C02F702061209305020E94991616
:102EE00080E092E00E94B61280910502D70115960B
:102EF0008C932FC00115110519F15F3F11F44F3F5D
:102F0000F9F0CD2CD1101CC08091CE012091CF01C1
:102F100036E0821709F45CC090E0389FF001399FD9
:102F2000F00D1124E053FE4F6181561306C06081FD
:102F3000461303C06281611103C001968770E9CF17
:102F4000CD2CDD2009F426C180910502816080939B
:102F50000502C12C1FC1651308C0341306C0D1106F
:102F600004C080910502D701C9C04D875E87DF8606
:102F7000702F198B088B6D2D89890E94021688236A
:102F8000E9F1DD20D9F120910502822F82958F7021
:102F900090E0029774F0809100029091010298876E
:102FA0008F8319861B870A872C87CE0107960E947C
:102FB000B61286E0F701A0E0B2E001900D928A958A
:102FC000E1F70E94A7160E949916CC24C394E2C090
:102FD000702F198B088B60E089890E94371B292F7D
:102FE00022952F7030E0223031050CF0C7C09F7061
:102FF00009F0C1C0805E883008F4CCC0C7010E94CF
:10300000B612E3CF0817190708F456C0F801E81BF9
:10301000F90BCF01883C910508F453C0C12C702FE7
:10302000198B088B6D2D89890E945916E0E0F2E01A
:1030300086E0DF011D928A95E9F70E949916AAC0E1
:10304000651314C0341312C0D11010C08091050252
:10305000F7018583C7010E94B61286E0E0E0F2E046
:10306000DF011D928A95E9F7CB2C94C04D875E87CE
:10307000DF86702F198B088B6D2D89890E940216AF
:10308000882309F4BBCFDD2009F4B8CF20910502D5
:10309000822F82958F7090E002970CF48ACF8091F6
:1030A0000002909101029A8389831B821D830C8305
:1030B0002E83CE0101967BCF80959095800F911F36
:1030C000A9CFCD2CDD2009F499CF65132EC0341380
:1030D0002CC02091050220FD1FC0822F82958F7089
:1030E000D9F0D70115962C9315978F3049F08F5F43
:1030F000982F9295907F822F8F70892B15968C93A5
:10310000C7010E94B61286E0F701A0E0B2E001908C
:103110000D928A95E1F791CF86E0F701A0E0B2E049
:1031200001900D928A95E1F735C04D875E87DF8665
:10313000702F198B088B6D2D89890E9402168111C1
:1031400038CF80910502816080930502C7010E94FB
:10315000B61220C0DD2009F451CF4D875E87DF868F
:10316000702F198B088B6D2D89890E940216882378
:1031700009F444CF1ECF81113DCF0CC0243031055E
:103180000CF03CCF9F7009F435CFF7019581907F0B
:1031900009F030CF8C2D61960FB6F894DEBF0FBECC
:1031A000CDBFDF91CF911F910F91FF90EF90DF90F6
:1031B000CF90BF9008951F93CF93DF93CDB7DEB725
:1031C0002C970FB6F894DEBF0FBECDBF4F83588744
:1031D00069877A878B879C87CE0107960E940217A2
:1031E000882369F08F8198852A853B85232BF1F10F
:1031F0009F3F09F063C08F3F09F060C037C086E091
:10320000FE013796DE01119601900D928A95E1F745
:103210006F817885EA85FB85309741F17F3F11F416
:103220006F3F21F12091CF0130E0C90101968770F5
:1032300099274091CE0150E08417950709F447C0C3
:1032400069837A83FD83EC8396E0929FD001939FFC
:10325000B00D1124A053BE4FFE01319601900D9286
:103260009A95E1F78093CF010E94781616E080913D
:10327000CE019091CF018917C1F1189FC00111248F
:1032800080539E4F0E940217882379F1E091CE016E
:103290001E9FF0011124E053FE4F40815181628155
:1032A0007381848195810E9468168091CE0190E09F
:1032B0000196877099278093CE01D9CF4F81588589
:1032C00069857A858B859C850E946816CFCF0E9480
:1032D000FE151092CF011092CE01E0E0F2E086E000
:1032E000DF011D928A95E9F7C1CF2C960FB6F894AD
:1032F000DEBF0FBECDBFDF91CF911F910895DF924A
:10330000EF92FF920F931F93CF93DF93FC01892BD2
:1033100009F48AC0E12CF12CDD24D394EF0121962D
:103320008491853709F461C058F4843708F04EC0A1
:10333000843008F06AC08130D1F0823071F174C0FD
:10334000883709F45DC050F4863709F455C08737D3
:1033500009F06AC08E2D0E946B1C54C09CE7980F28
:10336000903708F061C08F770E94801250C08F01A3
:103370000E5F1F4FFE01849190E2980F983050F439
:103380008770FD2D01C0FF0F8A95EAF78F2F0E94ED
:10339000711C14C00E94D61113C08F010E5F1F4F05
:1033A000FE01C49180E28C0F883060F4C7708D2DCF
:1033B00001C0880FCA95EAF70E94771C0E94981CEA
:1033C000E80125C08C2F0E948012FACF9F012E5F4A
:1033D0003F4FFE01C491CC2369F08FE99FE0019734
:1033E000F1F700C00000C150F6CF9F012E5F3F4FA4
:1033F000FE01F490E9010BC00E945B1CE82E07C09F
:103400000E946E1C0E94981C02C00E94D6118F2D33
:10341000882341F0EFE9FFE03197F1F700C00000A9
:103420008150F6CFFE017ACFDF91CF911F910F919E
:10343000FF90EF90DF90089560938602709387026B
:1034400080938802909389020C94EA1C08956093FB
:103450008A0270938B0280938C0290938D020C945D
:10346000E91C0F931F9300918A0210918B02209107
:103470008C0230918D02602B712B822B932B6093E9
:103480008A0270938B0280938C0290938D021F911D
:103490000F910C94E91C0F931F9300918A021091D5
:1034A0008B0220918C0230918D0260237123822344
:1034B000932360938A0270938B0280938C02909383
:1034C0008D021F910F910C94E91C0F931F93009193
:1034D0008A0210918B0220918C0230918D0260271C
:1034E00071278227932760938A0270938B028093BF
:1034F0008C0290938D021F910F910C94E91C60E057
:1035000070E0CB010C941C1A0F931F9341E050E024
:1035100060E070E08A019B0104C0000F111F221FB0
:10352000331F8A95D2F7C901B8011F910F910C94EE
:103530001C1A0F931F9341E050E060E070E004C05C
:10354000440F551F661F771F8A95D2F78091860218
:1035500090918702A0918802B09189028A019B0113
:10356000082B192B2A2B3B2BC901B8011F910F9156
:103570000C941C1A0F931F9341E050E060E070E040
:1035800004C0440F551F661F771F8A95D2F74095D8
:103590005095609570958091860290918702A091D8
:1035A0008802B09189028A019B01082319232A23EA
:1035B0003B23C901B8011F910F910C941C1A0F9362
:1035C0001F9341E050E060E070E004C0440F551FDD
:1035D000661F771F8A95D2F78091860290918702A5
:1035E000A0918802B09189028A019B0108271927BE
:1035F0002A273B27C901B8011F910F910C941C1A6F
:103600000F931F93009186021091870220918802E8
:1036100030918902602B712B822B932B1F910F917C
:103620000C941C1A0F931F9300918602109187022D
:103630002091880230918902602371238223932391
:103640001F910F910C941C1A0F931F9300918602E7
:10365000109187022091880230918902602771279A
:10366000822793271F910F910C941C1A08958F9213
:103670009F92AF92BF92DF92EF92FF920F931F93B0
:10368000CF93DF9300D000D01F92CDB7DEB76B830E
:103690007C838D838A018C819D81892B21F01F3F42
:1036A00029F44F3F19F480E090E04CC08B818823CF
:1036B000C9F180908A0290908B02A0908C02B09009
:1036C0008D028091860290918702A0918802B0912C
:1036D0008902882A992AAA2ABB2A8FE1E82EF12C8E
:1036E000D501C4010E2C04C0B695A7959795879572
:1036F0000A94D2F780FF07C0DE2CB8018E2D0E94FD
:10370000081E019729F481E0E81AF10848F7D12C46
:1037100088E0189FF0011124E00FF11DEA5FFD4FD2
:10372000D08209C088E0189FF0011124E00FF11D3C
:10373000EA5FFD4FD08009831A8369817A818D2DDC
:103740000E94081E0F900F900F900F900F90DF9126
:10375000CF911F910F91FF90EF90DF90BF90AF90AE
:103760009F908F90089590910A01992321F0909154
:103770000B01911109C020910C0130910D01F9014B
:1037800032969FEF40E030C0982F9695969596958B
:103790009F31A0F4E0910C01F0910D01E90FF11DB2
:1037A000877021E030E0A90102C0440F551F8A95BF
:1037B000E2F7CA019181892B818308959091B1022A
:1037C00090FF23C01F928F938FE294E09F938F937B
:1037D0000E942C060F900F900F900F9008959F3F1E
:1037E00039F04F5F4E3141F051915813F8CF0DC071
:1037F0005111F7CF942FF5CF9F3F39F0F901E90F21
:10380000F11D97FDFA9582830895089590910A011C
:10381000992321F090910B01911109C020910C0185
:1038200030910D01F9013296205E3F4F30C0982F44
:103830009695969596959F31A8F4E0910C01F0919C
:103840000D01E90FF11D877021E030E0A90102C0F0
:10385000440F551F8A95E2F7CA018095918189230B
:10386000818308959091B10290FF16C01F928F93AB
:1038700081E194E09F938F930E942C060F900F900C
:103880000F900F9008953196E217F30729F0908179
:103890009813F9CF1082F7CF089581E090E0E0917E
:1038A0000C01F0910D01E80FF91F10820196803292
:1038B0009105A9F708958091B00208959091B00202
:1038C000892B8093B002089580959091B00289234E
:1038D0008093B00208958093B00208951092B002D0
:1038E00008959091AF02892B8093AF02089580953F
:1038F0009091AF0289238093AF0208951092AF0296
:10390000089580938E02089510928E0208958091FA
:103910000C0190910D01FC0131969C01205E3F4FFE
:1039200080E0919191118F5FE217F307D1F708952D
:10393000E0910C01F0910D018091B0028083E09143
:103940000C01F0910D0190818091AF02892B808351
:1039500080918E02882361F0E0910C01F0910D01BD
:103960009081892B80830E94871C811110928E0286
:1039700080910C0190910D010C94E90F9093390105
:103980008093380108958295982F9C7C392F369525
:103990003695282F237344E0249FC0011124932FD0
:1039A000982B292F2A7A2695892F8575880F822BA7
:1039B00008950895CF93DF9300D000D01F92CDB724
:1039C000DEB70F900F900F900F900F90DF91CF9177
:1039D0000895089508950C9442118091C602843090
:1039E00021F11092B20220E488E190E00FB6F89441
:1039F000A895809360000FBE2093600083B7817FFD
:103A0000846083BF83B7816083BF7894889583B7D0
:103A10008E7F83BF0FB6F894A8958091600088616F
:103A200080936000109260000FBE0895CF930E94B3
:103A300094110E9478070E949511C0E08C2F0E947B
:103A4000FF07811104C0CF5FC031C1F701C081E021
:103A5000CF9108950E9405080C94FE151F920F92B5
:103A60000FB60F9211248F939F93AF93BF938091C2
:103A7000B202811113C08091B3029091B402A0915F
:103A8000B502B091B6024196A11DB11D8093B3025B
:103A90009093B402A093B502B093B602BF91AF91D8
:103AA0009F918F910F900FBE0F901F90189582E0FD
:103AB00084BD93E095BD9AEF97BD80936E00089505
:103AC0002FB7F8948091B3029091B402A091B502FF
:103AD000B091B6022FBF08952FB7F8946091B3024A
:103AE0007091B4028091B5029091B6022FBF0895F3
:103AF000CF92DF92EF92FF920F931F932FB7F8941C
:103B00004091B3025091B4026091B5027091B60237
:103B10002FBF6A017B01EE24FF248C0120E030E0FE
:103B2000C016D106E206F30610F4415051099A017D
:103B3000281B390BC9011F910F91FF90EF90DF9067
:103B4000CF9008951F920F920FB60F9211248F936A
:103B50009F93AF93BF938091B3029091B402A091D1
:103B6000B502B091B6020196A11DB11D8093B302BA
:103B70009093B402A093B502B093B602BF91AF91F7
:103B80009F918F910F900FBE0F901F9018950E94DC
:103B9000F60CF8942FEF87EA91E621508040904090
:103BA000E1F700C0000087E090EBDC018093CF02DA
:103BB0009093D002A093D102B093D2029CE088E10E
:103BC0000FB6F894A895809360000FBE90936000A4
:103BD000FFCF80E090E008950895E72FF0E090E1B6
:103BE000899FE00DF11D112483E0EE0FFF1F8A95E0
:103BF000E1F7E60FF11DEA50FF4F84910895E82F99
:103C0000F0E0EE0FFF1FEA58F0408591949108957F
:103C10000E94ED1D90E4980F903218F40E94FF1D51
:103C200008958D3B50F4883AA0F5853A28F5843004
:103C300000F5813009F49DC099C0883E98F4803E1B
:103C4000C0F48F3B09F092C00E94FE152FEF80E771
:103C500092E0215080409040E1F700C000000E94B7
:103C6000C71D84C0803F08F481C0282F30E0306534
:103C700082C0282F30E07FC0853A29F0863A31F0A3
:103C800023E830E478C021E830E475C022E830E46D
:103C900072C0883A61F1893A69F18A3A71F18B3AD6
:103CA00079F18C3A81F18D3A89F18E3A91F18F3A1E
:103CB00099F1813BA1F1803BA9F1823BB1F1833BBA
:103CC000B9F1843BC1F1853BC9F1863BD1F1873B1A
:103CD000D9F1883BE1F1893BE9F18A3BF1F18B3B7A
:103CE000F9F18C3B09F43FC020E034E444C022EEFB
:103CF00034E441C029EE34E43EC02AEE34E43BC053
:103D000025EB34E438C026EB34E435C023EB34E44F
:103D100032C024EB34E42FC027EB34E42CC02CEC6D
:103D200034E429C02DEC34E426C023E835E423C074
:103D30002AE835E420C022E935E41DC024E935E451
:103D40001AC021E236E417C023E236E414C024E2AC
:103D500036E411C025E236E40EC026E236E40BC09C
:103D600027E236E408C02AE236E405C020E030E06D
:103D700002C021E030E0C90108958091B90280FFBE
:103D80000BC06091110185E0689FB0011124759509
:103D90006795759567952BC081FF09C060911101EA
:103DA00085E0689FB00111247595679520C082FF5A
:103DB00007C06091110185E0689FB001112417C010
:103DC0009091BA029923D1F060911001961788F76B
:103DD0002091110185E0289F90011124929FA0015C
:103DE000939F500D112470E0CA010E9497266038FD
:103DF000710540F46115710539F002C065E070E0AD
:103E0000862F08958FE7089581E008958091B90283
:103E100080FF08C060910F0170E0759567957595FA
:103E2000679521C081FF06C060910F0170E0759514
:103E3000679519C082FF04C060910F0170E010C047
:103E40009091BA029923C1F060910E019617A0F7E4
:103E500080910F01899FC001112470E00E94972674
:103E60006038710528F46115710521F0862F0895D9
:103E70008FE7089581E0089561E070E0F4CF803F1E
:103E800021F40E94BD1E819504C0813F29F40E9447
:103E9000BD1E8093BD020895823F21F40E94BD1E85
:103EA000819504C0833F29F40E94BD1E8093BC020B
:103EB0000895893F19F40E94061F05C08A3F31F416
:103EC0000E94061F81958093BE0208958B3F21F4C6
:103ED0000E94061F819504C08C3F29F40E94061F92
:103EE0008093BF020895843F21F48091BB028160DA
:103EF00017C0853F21F48091BB02826011C0863FCC
:103F000021F48091BB0284600BC0873F21F4809133
:103F1000BB02886005C0883F31F48091BB0280619C
:103F20008093BB0208958D3F21F48091B902816096
:103F30000BC08E3F21F48091B902826005C08F3F93
:103F400029F48091B90284608093B9020895803F7A
:103F500039F48091BD0287FF6CC01092BD0269C028
:103F6000813F29F48091BD021816BCF362C0909184
:103F7000BC02823F29F497FF5CC01092BC0259C07A
:103F8000833F19F41916CCF354C0893F41F4809152
:103F9000BE0218160CF04DC01092BE024AC08A3FF5
:103FA00029F48091BE0287FF44C0F6CF8B3F39F4DD
:103FB0008091BF0287FF3DC01092BF023AC08C3F84
:103FC00029F48091BF021816BCF333C0843F21F45A
:103FD0008091BB028E7F17C0853F21F48091BB0288
:103FE0008D7F11C0863F21F48091BB028B7F0BC077
:103FF000873F21F48091BB02877F05C0883F31F461
:104000008091BB028F7E8093BB0213C08D3F21F451
:104010008091B9028E7F0BC08E3F21F48091B9024E
:104020008D7F05C08F3F29F48091B9028B7F8093EB
:10403000B9028091BC0281110EC08091BD02811134
:104040000AC08091BE02811106C08091BF02811119
:1040500002C01092BA0208958091B10283FF7EC01F
:1040600084E794E00E9493058091BB021F928F9396
:104070008FE694E09F938F930E942C068DE694E048
:104080000E9493058091BC02282F082E000C330B50
:104090003F938F938AE694E09F938F930E942C0620
:1040A00088E694E00E9493058091BD02282F082E97
:1040B000000C330B3F938F9385E694E09F938F938F
:1040C0000E942C0683E694E00E9493058091BE0234
:1040D000282F082E000C330B3F938F9380E694E03B
:1040E0009F938F930E942C068EE594E00E94930587
:1040F0008091BF02282F082E000C330B3F938F9323
:104100008BE594E09F938F930E942C0688E594E0C2
:104110000E9493058091BA021F928F9385E594E0E7
:104120009F938F930E942C0683E594E00E94930551
:104130008091B9021F928F9380E594E09F938F93B3
:104140000E942C068DE494E00E9493058DB79EB7E3
:104150004C960FB6F8949EBF0FBE8DBF8BEB92E0CE
:104160000E9432100E94601D9093B8028093B702A3
:1041700008951F93CF93DF938091B7029091B80277
:104180000E94781DAC019091BA02992321F02091F0
:10419000120130E006C0209113018AE0289F9001AF
:1041A00011244217530708F485C08091BC02C091C6
:1041B000BD02D091BE021091BF02811107C0C11192
:1041C00075C0D11173C0111171C074C09F3F19F037
:1041D0009F5F9093BA02181624F40E94BD1E80932C
:1041E000BC028091BC0287FF05C00E94BD1E819564
:1041F0008093BC021C1624F40E94BD1E8093BD0255
:104200008091BD0287FF05C00E94BD1E81958093ED
:10421000BD026091BC02662331F1C091BD02CC2386
:1042200011F1062E000C770B880B990B0E9492253A
:1042300023E333E343E35FE30E94F6250E945A251C
:104240006093BC026C2FCC0F770B880B990B0E94EC
:10425000922523E333E343E35FE30E94F6250E94C4
:104260005A256093BD021D1624F40E94061F8093F8
:10427000BE028091BE0287FF05C00E94061F819585
:104280008093BE02111624F40E94061F8093BF0281
:104290008091BF0287FF05C00E94061F8195809311
:1042A000BF02DF91CF911F910C942C209F3F09F00A
:1042B0008FCF97CFDF91CF911F910895EBEBF2E075
:1042C00085E0DF011D928A95E9F71092BA021092FB
:1042D000B902089587E996E00E9493051F9281E054
:1042E0008F931F9285E08F9389E496E09F938F933D
:1042F0000E942C060F900F900F900F900F900F9030
:1043000008958330E9F128F4813061F0823009F1B9
:104310000895853009F462C008F449C0863009F474
:1043200074C0089580911301262F30E0280F311DAD
:104330002F3F310524F4680F6093130103C08FEF02
:1043400080931301809113011F928F9382E895E06F
:1043500072C080911201262F30E0280F311D2F3FAF
:10436000310524F4680F6093120103C08FEF80932E
:104370001201809112011F928F9380E795E05BC03C
:1043800080911101262F30E0280F311D2F3F31057C
:1043900024F4680F6093110103C08FEF8093110123
:1043A000809111011F928F938DE595E044C080911B
:1043B0001001262F30E0280F311D2F3F310524F446
:1043C000680F6093100103C08FEF809310018091FC
:1043D00010011F928F9388E495E02DC080910F010A
:1043E000262F30E0280F311D2F3F310524F4680FB0
:1043F00060930F0103C08FEF80930F0180910F0135
:104400001F928F938FE295E016C080910E01262FA8
:1044100030E0280F311D2F3F310524F4680F6093E1
:104420000E0103C08FEF80930E0180910E011F9249
:104430008F9384E195E09F938F930E942C060F90B9
:104440000F900F900F900895833081F128F4813000
:1044500059F08230D1F00895853009F449C0B8F19F
:10446000863009F456C0089580911301681720F42E
:10447000861B8093130102C01092130180911301D7
:104480001F928F9385E095E054C0809112016817C8
:1044900020F4861B8093120102C0109212018091B9
:1044A00012011F928F9383EF94E043C0809111011A
:1044B000681720F4861B8093110102C0109211012D
:1044C000809111011F928F9380EE94E032C0809111
:1044D0001001681720F4861B8093100102C010920F
:1044E0001001809110011F928F938BEC94E021C0FA
:1044F00080910F01681720F4861B80930F0102C082
:1045000010920F0180910F011F928F9382EB94E024
:1045100010C080910E01681720F4861B80930E0155
:1045200002C010920E0180910E011F928F9387E9B5
:1045300094E09F938F930E942C060F900F900F9002
:104540000F900895CF93C82F1F928F938CE997E017
:104550009F938F930E942C0681E090E0A0E0B0E052
:10456000BC01CD0104C0660F771F881F991FCA9533
:10457000D2F70E94271A0F900F900F900F90CF91B3
:104580000C94FE15CF938732A8F58E3108F02BC11D
:10459000803109F49FC0F8F4873009F464C0A8F4AE
:1045A000863009F024C18091B102817F8E7F809393
:1045B000B10281EA97E00E94930587E79AE00E94A2
:1045C000930581E08093C1024CC08B30F1F18E30B5
:1045D00009F46CC00CC1863109F4B0C020F48131FB
:1045E00009F4EDC004C1893109F491C08B3109F49B
:1045F00049C0FDC0883349F150F4893209F4F1C053
:10460000853309F4EEC0873209F0F1C0EAC0833483
:1046100009F4E7C028F48A3308F4E9C08953E4C0F8
:10462000883409F0E4C00E94FE1586E69AE00E94F4
:1046300093052FEF83ED90E3215080409040E1F708
:1046400000C000000E94C71D0CC088EC97E05CC051
:104650008DE49AE00E9493058091B102816080937D
:10466000B102C1E0C9C08091B102C82FC17080FF02
:10467000EFCF89E59AE00E9493058091B102817F96
:104680008E7F3DC09091B10291FBCC27C0F981E0B3
:10469000C827892FC0FB81F98093B102CC2319F080
:1046A00080E49AE027C082E39AE02EC09091B102A4
:1046B00092FBCC27C0F981E0C827892FC0FB82F983
:1046C0008093B102CC2319F083E29AE013C083E116
:1046D0009AE01AC09091B10293FBCC27C0F981E017
:1046E000C827892FC0FB83F98093B102CC2351F0F6
:1046F00087E09AE00E9493058091B10281608093E7
:10470000B1027AC08AEF99E00E949305AACF8BEE9E
:1047100099E00E94930589EC99E00E94930585E851
:1047200099E00E9493058EE599E00E94930584E24A
:1047300099E00E94930586EF98E0E6CF88EE98E036
:104740000E9493050E94DD0F1F928F938EEC98E0DC
:104750009F938F930E942C0680910A011F928F9342
:1047600087EB98E09F938F930E942C068091B6016F
:104770001F928F9384EA98E09F938F930E942C0658
:1047800080910B011F928F9381E998E09F938F9303
:104790000E942C060E946C1D9F938F937F936F93B2
:1047A0008AE798E09F938F930E942C068DB79EB75F
:1047B00046960FB6F8949EBF0FBE8DBF52CF0E9493
:1047C000FE15C0910B0181E0C827C0930B01CC23DB
:1047D00029F080E798E00E9493050EC085E698E0F6
:1047E00093CF80E001C08D510E94A2223ACF83E690
:1047F00098E00E949305C0E08C2FCF91089580E04F
:10480000089580E00895CF93C82F8091C102813030
:1048100079F020F0823009F44DC044C1E0910C01E0
:10482000F0910D0180818152823008F03DC108C0B5
:10483000E0910C01F0910D0180818152823060F491
:104840008C2F0E94FF23811104C08C2F0E94C22252
:104850002FC081E090E02CC08C2F0E940124811198
:1048600026C0C431E1F070F4CB3081F0C031D1F416
:104870000E946A2184E997E00E94930582E0809378
:10488000C10215C0C93259F0C83361F481EA97E01A
:104890000E94930588E997E00E94930508C0109252
:1048A000C10204C182E997E00E949305FFC081E044
:1048B0008170FEC0C43228F5CE3108F0C1C0CB30C3
:1048C000A1F1D0F4C73009F0D3C08EE18093130179
:1048D00082E3809312018AE08093110184E1809346
:1048E000100188E080930F0188E280930E0188E335
:1048F00096E00E949305BFC0C33149F1C431C1F0B5
:10490000B7C0CB3409F4A9C028F4C93289F0C83340
:1049100061F0AEC0C13509F49EC0C23509F499C03A
:10492000CE3409F0A5C06AE09EC00E946A21A3C0EF
:104930008091C002882319F01092C0029CC085E4C7
:1049400096E00E94930581E08093C102B1C08FE19F
:1049500096E00E9493058DE096E00E949305809179
:1049600013011F928F938AE096E09F938F930E948A
:104970002C0688E096E00E94930586EF95E00E9461
:104980009305809112011F928F9383EF95E09F937F
:104990008F930E942C0681EF95E00E94930582EE92
:1049A00095E00E949305809111011F928F938FEDE6
:1049B00095E09F938F930E942C068DED95E00E94C9
:1049C00093058CEC95E00E949305809110011F9255
:1049D0008F9389EC95E09F938F930E942C0687EC30
:1049E00095E00E94930582EB95E00E9493058091EB
:1049F0000F011F928F938FEA95E09F938F930E94F0
:104A00002C068DEA95E00E94930586E995E00E94C8
:104A1000930580910E011F928F9383E995E09F93F8
:104A20008F930E942C0681E995E00E9493058DB733
:104A30009EB748960FB6F8949EBF0FBE8DBF1BC0A1
:104A4000CE51EC2FF0E0E25DFE4F80818093C002FA
:104A500012C061E003C061E006C06AE08091C0025C
:104A60000E94812108C08091C0020E94242203C0BC
:104A700086E396E013C08091C002882369F01F92FC
:104A80008F9380E396E09F938F930E942C060F9064
:104A90000F900F900F9004C08DE296E00E94930556
:104AA00081E006C01092C10280E002C080E000CF29
:104AB000CF9108950E9461256894B1110C94F0255E
:104AC00008950E94D52588F09F5798F0B92F99270F
:104AD000B751B0F0E1F0660F771F881F991F1AF0E9
:104AE000BA95C9F714C0B13091F00E94EF25B1E03A
:104AF00008950C94EF25672F782F8827B85F39F039
:104B0000B93FCCF3869577956795B395D9F73EF481
:104B100090958095709561957F4F8F4F9F4F089529
:104B2000E89409C097FB3EF4909580957095619547
:104B30007F4F8F4F9F4F9923A9F0F92F96E9BB27FD
:104B40009395F695879577956795B795F111F8CF79
:104B5000FAF4BB0F11F460FF1BC06F5F7F4F8F4FE4
:104B60009F4F16C0882311F096E911C0772321F0DA
:104B70009EE8872F762F05C0662371F096E8862F72
:104B800070E060E02AF09A95660F771F881FDAF7C9
:104B9000880F9695879597F9089557FD9058440F7B
:104BA000551F59F05F3F71F04795880F97FB991F8C
:104BB00061F09F3F79F08795089512161306140649
:104BC000551FF2CF4695F1DF08C0161617061806D6
:104BD000991FF1CF86957105610508940895E894B1
:104BE000BB2766277727CB0197F908950E940926EE
:104BF0000C947A260E946C2638F00E94732620F0CE
:104C0000952311F00C9463260C94692611240C94BE
:104C1000F0250E94CD2570F3959FC1F3950F50E0CC
:104C2000551F629FF001729FBB27F00DB11D639F5E
:104C3000AA27F00DB11DAA1F649F6627B00DA11D04
:104C4000661F829F2227B00DA11D621F739FB00DAA
:104C5000A11D621F839FA00D611D221F749F33271A
:104C6000A00D611D231F849F600D211D822F762FB3
:104C70006A2F11249F5750409AF0F1F088234AF090
:104C8000EE0FFF1FBB1F661F771F881F91505040FC
:104C9000A9F79E3F510580F00C9463260C94F025F3
:104CA0005F3FE4F3983ED4F3869577956795B79583
:104CB000F795E7959F5FC1F7FE2B880F911D96959D
:104CC000879597F9089597F99F6780E870E060E00D
:104CD00008959FEF80EC089500240A941616170695
:104CE00018060906089500240A94121613061406DD
:104CF00005060895092E0394000C11F4882352F040
:104D0000BB0F40F4BF2B11F460FF04C06F5F7F4FF7
:104D10008F4F9F4F0895991B79E004C0991F9617F4
:104D200008F0961B881F7A95C9F78095089597FB20
:104D3000072E16F4009407D077FD09D00E94B12603
:104D400007FC05D03EF4909581959F4F089570958E
:104D500061957F4F0895EE0FFF1F0590F491E02DB0
:104D60000994AA1BBB1B51E107C0AA1FBB1FA617B2
:104D7000B70710F0A61BB70B881F991F5A95A9F704
:0E4D800080959095BC01CD010895F894FFCF69
:104D8E000E08FF08DC08A808740801018F02280825
:104D9E00140A321E404D36223979032C03F602D402
:104DAE00029B020E02270240025902790200010202
:084DBE000304050607080900C3
:00000001FF
